:100000000C9446000C9468000C9468000C946800F2
:100010000C9468000C9468000C9468000C946800C0
:100020000C9468000C9468000C9468000C946800B0
:100030000C9468000C9468000C9468000C946800A0
:100040000C9468000C9468000C9468000C94680090
:100050000C9468000C9468000C9468000C94680080
:100060000C9468000C9468000C9468000C94680070
:100070000C9468000C9468000C9468000C94680060
:100080000C9468000C9468000C94680011241FBE46
:1000900020E0A89521BD20E025BF2FEF2DBF20E156
:1000A0002EBFE2E6F2E030E0A0E0B1E021E03BBFAD
:1000B00002C007900D92A030B207D9F7A0E0B1E0DE
:1000C00021E001C01D92A030B207E1F70C9482003C
:1000D0000C946A001895880F991F1816190614F4C5
:1000E0000197F1F70895CF93DF93181619063CF4A2
:1000F000EC0188EE93E00E946B002197D1F7DF912D
:10010000CF910895C5E3D0E1DEBFCDBF95E6492E7E
:10011000512C4C0E5D1E14E6D2011D921A95E9F782
:100120000FEF0ABB07BB04BB11BA02B90093610011
:100130001E010894211C311C320103E610E0600E00
:10014000711EC753DF4F48825982C95CD040CC240E
:10015000DD24460156018201710130B3F70131936C
:100160007F01D8012D918D0128BB81E090E00E9494
:100170007300601671068CF789818170992720E0E1
:1001800030E0F101892BA9F18191817099272F5FCE
:100190003F4F24363105B4F354E6D2011D925A95EF
:1001A000E9F7CC0CDD1CC601B4010E940A014B0129
:1001B000C4016CE070E00E940A016B01C60141E0DD
:1001C00050E0BA01C753DF4FE881F981C95CD040E4
:1001D0009F012D593F4F4083019729F031962E17EB
:1001E0003F07CCF7B4CFC6015B01A41AB50AA5013D
:1001F000F5CFE080E0FEC8CFA114B10441F0A90121
:100200004A195B09C40ED51E0894811C911C590122
:10021000BBCFFFCF97FB092E07260AD077FD04D06E
:100220000CD006D000201AF4709561957F4F089588
:10023000F6F7909581959F4F0895AA1BBB1B51E13E
:1002400007C0AA1FBB1FA617B70710F0A61BB70B46
:10025000881F991F5A95A9F780959095BC01CD01EB
:020260000895FF
:00000001FF
